:1000000010C02AC029C028C027C026C025C024C0CF
:1000100023C022C021C020C01FC01EC01DC01CC0E4
:100020001BC011241FBECFE5D1E0DEBFCDBF10E065
:10003000A0E6B0E0E4E5F1E002C005900D92A03644
:10004000B107D9F720E0A0E6B0E001C01D92A536C7
:10005000B207E1F70ED07CC0D3CF369A3699FECFE7
:1000600084B195B1089582E087B993E896B981B9D2
:100070000895D39AD49AD698F6DF1092600011E0D2
:10008000C4E6D0E0CE9947C02FE73AE146E02150E0
:1000900030404040E1F700C00000CE993CC0809164
:1000A0006000812780936000CE9BFECF34C0EFE3D9
:1000B000FDE023E0E150F0402040E1F700C0000007
:1000C000019620916100309162002817390778F776
:1000D00027C0EFE4F3EC3197F1F700C00000019680
:1000E00020916100309162002817390790F7CACF3C
:1000F000DB98DC9AC7CFDB9AB0DF909364008093E3
:100100006300BE0111D07093620060936100DC98BF
:1001100080E090E0CCCF80916000882349F3EBCF62
:10012000DC9A80E090E0D5CFAA1BBB1B51E107C051
:10013000AA1FBB1FA617B70710F0A61BB70B881F77
:10014000991F5A95A9F780959095BC01CD01089506
:04015000F894FFCF51
:00000001FF
